BL51 BANKED LINKER/LOCATER V5.03                                                        06/14/2006  12:20:41  PAGE 1


BL51 BANKED LINKER/LOCATER V5.03, INVOKED BY:
C:\KEIL\C51\BIN\BL51.EXE STARTUP.obj, main.obj TO hblinkLED RAMSIZE (256) CODE (0X0000-0X1FFF)


MEMORY MODEL: SMALL


INPUT MODULES INCLUDED:
  STARTUP.obj (?C_STARTUP)
  main.obj (MAIN)


LINK MAP OF MODULE:  hblinkLED (?C_STARTUP)


            TYPE    BASE      LENGTH    RELOCATION   SEGMENT NAME
            -----------------------------------------------------

            * * * * * * *   D A T A   M E M O R Y   * * * * * * *
            REG     0000H     0008H     ABSOLUTE     "REG BANK 0"
            DATA    0008H     0001H     UNIT         _DATA_GROUP_
            IDATA   0009H     0001H     UNIT         ?STACK

            * * * * * * *   C O D E   M E M O R Y   * * * * * * *
            CODE    0000H     0003H     ABSOLUTE     
                    0003H     0008H                  *** GAP ***
            CODE    000BH     0003H     ABSOLUTE     
                    000EH     07F2H                  *** GAP ***
            CODE    0800H     001BH     UNIT         ?PR?TMR0?MAIN
            CODE    081BH     0011H     UNIT         ?PR?TMR0INIT?MAIN
            CODE    082CH     000CH     UNIT         ?C_C51STARTUP
            CODE    0838H     0007H     UNIT         ?PR?MAIN?MAIN



OVERLAY MAP OF MODULE:   hblinkLED (?C_STARTUP)


SEGMENT                          DATA_GROUP 
  +--> CALLED SEGMENT          START    LENGTH
----------------------------------------------
?C_C51STARTUP                  -----    -----
  +--> ?PR?MAIN?MAIN

?PR?MAIN?MAIN                  -----    -----
  +--> ?PR?TMR0INIT?MAIN

*** NEW ROOT ***************************************************

?PR?TMR0?MAIN                  0008H    0001H



SYMBOL TABLE OF MODULE:  hblinkLED (?C_STARTUP)

  VALUE           TYPE          NAME
  ----------------------------------

BL51 BANKED LINKER/LOCATER V5.03                                                      06/14/2006  12:20:41  PAGE 2


  -------         MODULE        ?C_STARTUP
  C:082CH         SEGMENT       ?C_C51STARTUP
  I:0009H         SEGMENT       ?STACK
  C:0000H         PUBLIC        ?C_STARTUP
  D:00E0H         SYMBOL        ACC
  D:00F0H         SYMBOL        B
  D:0083H         SYMBOL        DPH
  D:0082H         SYMBOL        DPL
  N:0000H         SYMBOL        IBPSTACK
  N:0100H         SYMBOL        IBPSTACKTOP
  N:0080H         SYMBOL        IDATALEN
  C:082FH         SYMBOL        IDATALOOP
  N:0000H         SYMBOL        PBPSTACK
  N:0000H         SYMBOL        PBPSTACKTOP
  N:0000H         SYMBOL        PDATALEN
  N:0000H         SYMBOL        PDATASTART
  N:0000H         SYMBOL        PPAGE
  N:0000H         SYMBOL        PPAGEENABLE
  D:00A0H         SYMBOL        PPAGE_SFR
  D:0081H         SYMBOL        SP
  C:082CH         SYMBOL        STARTUP1
  N:0000H         SYMBOL        XBPSTACK
  N:0000H         SYMBOL        XBPSTACKTOP
  N:0000H         SYMBOL        XDATALEN
  N:0000H         SYMBOL        XDATASTART
  C:0000H         LINE#         92
  C:082CH         LINE#         99
  C:082EH         LINE#         100
  C:082FH         LINE#         101
  C:0830H         LINE#         102
  C:0832H         LINE#         151
  C:0835H         LINE#         155
  -------         ENDMOD        ?C_STARTUP

  -------         MODULE        MAIN
  C:0000H         SYMBOL        _ICE_DUMMY_
  D:0090H         PUBLIC        P1
  D:00A0H         PUBLIC        P2
  D:00B0H         PUBLIC        P3
  B:00A8H.7       PUBLIC        EA
  D:00A8H         PUBLIC        IE
  D:00B8H         PUBLIC        IP
  C:0838H         PUBLIC        main
  D:0098H         PUBLIC        SCON
  D:0089H         PUBLIC        TMOD
  D:0088H         PUBLIC        TCON
  B:00A8H.1       PUBLIC        ET0
  D:008CH         PUBLIC        TH0
  D:008AH         PUBLIC        TL0
  B:00A0H.0       PUBLIC        LED
  B:0088H.4       PUBLIC        TR0
  C:0800H         PUBLIC        Tmr0
  D:00C8H         PUBLIC        T2CON
  D:00D0H         PUBLIC        PSW
  C:081BH         PUBLIC        Tmr0Init
  -------         PROC          TMR0
  -------         DO            
BL51 BANKED LINKER/LOCATER V5.03                                                      06/14/2006  12:20:41  PAGE 3


  D:0008H         SYMBOL        cnt
  -------         ENDDO         
  C:0800H         LINE#         52
  C:0804H         LINE#         55
  C:0806H         LINE#         56
  C:0810H         LINE#         57
  C:0813H         LINE#         58
  C:0816H         LINE#         60
  -------         ENDPROC       TMR0
  -------         PROC          TMR0INIT
  C:081BH         LINE#         79
  C:081BH         LINE#         80
  C:081BH         LINE#         82
  C:081EH         LINE#         83
  C:0821H         LINE#         85
  C:0824H         LINE#         86
  C:0827H         LINE#         88
  C:0829H         LINE#         89
  C:082BH         LINE#         90
  -------         ENDPROC       TMR0INIT
  -------         PROC          MAIN
  C:0838H         LINE#         99
  C:0838H         LINE#         100
  C:0838H         LINE#         101
  C:083BH         LINE#         102
  C:083DH         LINE#         104
  C:083DH         LINE#         105
  C:083DH         LINE#         107
  -------         ENDPROC       MAIN
  -------         ENDMOD        MAIN

******************************************************************************
* RESTRICTED VERSION WITH 0800H BYTE CODE SIZE LIMIT; USED: 004DH BYTE ( 3%) *
******************************************************************************

Program Size: data=10.0 xdata=0 code=69
LINK/LOCATE RUN COMPLETE.  0 WARNING(S),  0 ERROR(S)
